:0300000002337C4C
:0C337C0078FFE4F6D8FD7581790233C3B8
:100E74000A53746172743A20004950436F6E6E6570
:100E840063745245510A004950436F6E6E65637432
:100E9400003E432C562C43432CC0E4E0EFF2E5F033
:100EA40020D1E8EDEAEEEC49500A003E432C4D41D6
:100EB400432C25303262583A25303262583A253074
:100EC4003262583A25303262583A25303262583A02
:100ED40025303262582C4D414320E0E4F0E5F10A1C
:100EE400003E432C5645522C20332E3020EEF22067
:100EF40025732025732CC2E5F0F1E8FF204950202A
:100F0400ECEEE4F3EBFF0A004A756C203139203231
:100F14003030370031303A32343A3037003E432CE7
:100F24004C442C50524F473A20202020202020208F
:100F340020202020202020202020202020202020AD
:100F4400202020202020202020202020202020209D
:100F5400202020202020202020202020202020208D
:100F6400202020202020202020202020202CC4E00D
:100F7400F2E020EFF0EEF8E8E2EAE828F4E0E9EB4A
:100F8400290A003E2A2C312CCEF1EDEEE2EDFBE5F0
:100F940020EFE0F0E0ECE5F2F0FB20F1E5F2E5E231
:100FA400EEE3EE20E8EDF2E5F0F4E5E9F1E00A0025
:100FB4003E412C4130312C2562752E2562752E253B
:100FC40062752E2562752C495020E0E4F0E5F1208D
:100FD400E0E4E0EFF2E5F0E00A003E412C4130327B
:100FE4002C2562752E2562752E2562752E25627557
:100FF4002C495020E0E4F0E5F120EEF1ED2E20F153
:10100400E5F0E2E5F0E00A003E412C4130332C25C6
:1010140062752E2562752E2562752E2562752C4902
:101024005020E0E4F0E5F120F0E5E72E20F1E5F0D2
:10103400E2E5F0E00A003E412C4130342C25627593
:101044002E2562752E2562752E2562752CCCE0F155
:10105400EAE020F1E5F2E80A003E412C4130352C6B
:101064002562752E2562752E2562752E2562752CD6
:10107400D8EBFEE70A003E532C4130362C2562752E
:101084002CC2F0E5ECFF20EEE6E8E42E20EAE2E8EC
:10109400F2E0EDF6E8E820282A3130ECF1290A00E4
:1010A4003E2A2C312CC4EEEF2E20EFE0F0E0ECE5EC
:1010B400F2F0FB20F1E5F2E5E2EEE3EE20E8EDF2FA
:1010C400E5F0F4E5E9F1E00A003E422C5330312C1E
:1010D4002562752CC6E4E0F2FC20E7E0EFF0EEF1C7
:1010E400E020F1EEE5E4E8EDE5EDE8FF20EEF220A6
:1010F400F1E5F0E2E5F0E00A003E422C5330322CF8
:101104002562752C43E2FFE7FC20F120F1E5F0E2D3
:10111400E5F0EEEC20EDE520EFEEE4E4E5F0E6E8C2
:10112400E2E0F2FC0A003E422C5330332C25627577
:101134002CCFE5F0E5E7E0EFF3F1EA20EFF0E8206B
:10114400EFEEF2E5F0E520F1E2FFE7E820F120F12F
:10115400E5F0E2E5F0EEEC0A003E422C5330342C8C
:101164002562752CCDE5F220EFE5F0E5E4E0F7E843
:1011740020E4E8E0E3EDEEF1F2E8EAE820E220F131
:10118400E5F0E2E5F00A003E422C5330352C2562AE
:10119400752CCAE0EDE0EB20F8E8F0EEEAEEE2E5CB
:1011A400F8E0F2E5EBFCEDEEE3EE20EEE1ECE5ED4C
:1011B400E00A003E532C5330362C25303262582539
:1011C4003032625825303262582530326258253028
:1011D40032625825303262582C4D414320E0E4F00D
:1011E400E5F120F8E8F0EEEAEEE2E5F8E0F2E5EB0E
:1011F400FCEDEEE3EE20EEE1ECE5EDE00A003E4529
:101204004E440A0044756D70582020202020303050
:10121400203031203032203033203034203035201B
:1012240030362030372030382030392030412030DB
:10123400422030432030442030452030460A003AD2
:1012440020000A0044756D70442020202020303096
:1012540020303120303220303320303420303520DB
:10126400303620303720303820303920304120309B
:10127400422030432030442030452030460A004587
:101284007272206B657900526420656570726F6DAF
:101294000A005264204D454D0A00526420436F6495
:1012A400650A0044656275674950204F4E0A004440
:1012B400656275674950204F46460A004465627569
:1012C4006755736572204F6E0A00446562756755F1
:1012D400736572204F46460A0044656275674D7314
:1012E40067204F6E0A0044656275674D7367204F2F
:1012F40046460A00436F6E666967206C6F636B2114
:101304000A00577220656570726F6D0A0020536180
:10131400766520656570726F6D210A0045727220D2
:101324004D414321004C6F61643E3E002A003C4124
:1013340030313D003C4130323D003C4130333D00D2
:101344003C4130343D003C4130353D003C41303679
:101354003D004E4F4950004C494E4B434F4E545262
:10136400005452415353004652004E4F4C494E4B89
:1013740000494E49004E4F4449414700003C21007A
:101384003C5330313D003C5330323D003C5330330C
:101394003D003C5330343D003C5330353D003C531C
:1013A40030363D00FF1356FF135BFF1365FF136BCD
:0C13B400FF136EFF1375FF1379FF138009
:063B3B00010B000109006E
:103C9A00C2AFC28E758900438910758BFF758DB7C7
:073CAA00D2ABD28ED2AF2293
:03001B0002325559
:10325500C0E0C083C082C0D0C2AFC28E758BFF757F
:103265008DB720060675A61E75A6E10509D202E5ED
:103275000B6002050BE50AD394014002150A050E01
:10328500E50E540F704AD20DE50E543F7014D2006E
:1032950090668DE0600C04F0E0D394B44004C2AFB6
:1032A50080FE906688E0600204F0906104E06002B0
:1032B50014F090668EE0D394014003E014F03005DD
:1032C50002050CE50DD394644004D2068002050D79
:1032D500E508D3940140021508D28ED2AFD0D0D0E4
:0632E50082D083D0E0322C
:10086900C291C290D2B5C20A7D027C007F07123CB8
:100879002E8F5AE55A646060097D017F60123BE65C
:10088900D20AE4FDFC7F0B123C2E8F5AE55A30E662
:10089900097D04E4FF123C0AD20A7D017C007F072E
:1008A900123C2E8F5AE55A7008FD7FFF123BE6D2A3
:1008B9000A300A03126000C2AFC288C2A8C2AA12D3
:1008C9003611906341E0B4FA09A3E064CE700302E3
:1008D9000960E4F55A7439255AF582E43463F583DD
:1008E900E4F0055AE55AB443EC90634174FAF0A375
:1008F90074CEF0A374CCF0906347740AF0E4A3F0CB
:10090900A304F0A3F090634C7403F0A374CCF090AB
:10091900633D74FFF0A3F0A3F0E4A3F0906358746F
:1009290005F0E4F55AE55A2401FFE433FE7439254C
:100939005AF582E43463F583E0FD123C81055AE5FA
:100949005AC3944340DFE4F5A775A61E75A6E19046
:100959007FF0F0A3F080FED2AF90634C7403F0A354
:1009690074CCF0E490634BF0122D97EF60031220E2
:10097900AEC2B51237FEC206123A01906358E0C3FF
:10098900940350037403F0D20CD20BD20AD29320F1
:100999000A077E0E7F74122E7DE4906578F0123C72
:1009A9009AC2AFA37408F09062B77424F0E4A3F07C
:1009B900906341E09062B9F0906342E09062BAF0CE
:1009C900906343E09062BBF0906344E09062BCF0B6
:1009D900906345E09062BDF0906346E09062BEF09E
:1009E900750A01E490657AF0C207C208D2AF75A70B
:1009F9000775A61E75A6E1200A18AF5AFE7D0312D7
:100A09002F5EE4FF12310C7E637F78E4FB7D0112D7
:100A1900303890668DE060037401F0E4906104F071
:100A2900A37455F0A37481F0E4F50CE4F50D90611D
:100A390004E07003121B6590668EE0B4011190808A
:100A4900007410F0E490668EF0D20AD20BD20C90AA
:100A59008008E0F55A30E405D2077410F0E55A3001
:100A6900E508D2099080087420F0E55A30E608D2EA
:100A7900089080087440F0E50CD3940340239080DB
:100A890002E4F0908001F0908000F0E50CD3940628
:100A9900400FE4F50CC20390657AF0750A01123A29
:100AA900019080A0E0700312370A9080B8E07003CB
:100AB9001237849080D0E070031238E1908000E012
:100AC9007013300710122C93906334EFF0D3940015
:100AD9004003120026908002E07006908000E060DA
:100AE90005D205020A34C205E4F50C906104E06000
:100AF90003020A3430091212290E906334EFF0D33D
:100B090094004005E0FF123CC0200803020C8A1241
:100B19002799906334EFF07003020A3490668DE0F0
:100B290060037401F0906378E054BF247F7003027E
:100B39000BF6147003020BD724026003020C292060
:100B49000A077E0E7F7D122E7D300E792003769066
:100B59006350E07006906354E0605B906684E0FF48
:100B6900906350E0B50724906685E0FE906351E0FC
:100B7900B50618906686E0FE906352E0B5060C90C3
:100B89006687E0FE906353E06E602B906354E06FDC
:100B99007033906685E0FF906355E0B5072790664E
:100BA90086E0FF906356E0B5071B906687E0FF90EB
:100BB9006357E0B5070F90657A7401F0123CC2756E
:100BC9000A01020C8A90668474FFF0020C8A90660E
:100BD9007CE0FF90637AE06F6003020C8A90667C88
:100BE900E004F0E4F50A906578F0020C8A3003031A
:100BF900020C8A906347E07003020A3412001ED285
:100C090003E4F50A906578F090668804F0E490664C
:100C19007BF0A3F0200A6A7E0E7F8B122E7D806105
:100C2900300352906378E020E74B90637AE0FF90BD
:100C3900667BE0FE6F600D906683E07007EE146FCF
:100C4900703F801390667BE004F0906334E0FFD33B
:100C590094044003123CBC9060007482F0A37401B8
:100C6900F090637AE0906002F07E607F007D03126D
:100C7900368F020A34300E0920030690668474FF09
:100C8900F0200303020D3FE50A706B1231B6EF60E5
:100C9900207E647F78906479E02404FD12368F9079
:100CA9006683E06003020A34906358E0F50A020A99
:100CB90034906688E0D3943C403C906683E070367B
:100CC90090668804F09062B6E0702B123CC1E49003
:100CD9006478F0A37412F090667CE090647AF0A3D3
:100CE90074FDF090610763A20190647C63A2017FA7
:100CF9001212237C809B123CB1EF60159060007446
:100D090083F0E4A3F07E607F007D0212368F020A31
:100D190034E50A64016003020A34906578E004F05E
:100D2900E0C394055003020C9AC203E490657AF07B
:100D3900123CC2020A34E50A64016003020A3490D3
:100D4900657AE014604024FE603C147003020E27AB
:100D590024046003020A34E4F50C200E1390657A2A
:100D69007404F0906578E05401F0750A01020A34C0
:100D7900E490657AF090657804F0750AC890668405
:100D890074FFF0020A34906684E07003020E169034
:100D990064787480F090647A7401F0E4A3F0A30499
:100DA900F0A37430F0A3747BF0E4F55A747F255AEC
:100DB900F582E43464F583747DF07480255AF582F4
:100DC900E43464F583E4F0E55A2407906479F07C0F
:100DD900667D8490634CE0FAA3E0FB7F0212348DB8
:100DE9007E647F78E55A2409FD12368F906683E088
:100DF900601B12001ED203E4F50A906578F0906634
:100E09008804F0E490667BF0A3F0020A3490657AD6
:100E19007404F0906358E02432F50A020A34908091
:100E2900027410F0750A03906578E06401FFF09090
:100E3900657A7401F0EF7019906354E06013FCA3B4
:100E4900E0FDA3E0FEA3E0FF906684121F70020A92
:100E590034906350E0FCA3E0FDA3E0FEA3E0FF9023
:0A0E69006684121F70020A3480FE36
:010E7300225C
:10002600906379E0B444047F0180027F0090637896
:10003600E0B447047E0180027E00EE5F604A906372
:1000460041E090637AF0906342E090637BF09063C6
:1000560043E090637CF0906344E090637DF09063AE
:1000660045E090637EF0906346E090637FF0906396
:10007600797452F09062B063A2019080A863A201E5
:100086007F0612237C02085F906334E0C394085015
:1000960003020868906341E0FF90637AE06F6003B3
:1000A600020868906342E0FF90637BE06F600302A2
:1000B6000868906343E0FF90637CE06F600302088A
:1000C60068906344E0FF90637DE06F600302086818
:1000D600906345E0FF90637EE06F600302086890DE
:1000E6006346E0FF90637FE06F60030208689063F9
:1000F60079E0B444159062B0E0B4FF0E63A20190BB
:1001060080A863A2017F0612237C90668DE06003BF
:100116007401F090668E7464F09063797452F09076
:100126006378E0646D60030202A37BFF7A0E799523
:1001360012186B7BFF7A0E79AF906341E0F564A3EA
:10014600E0F565A3E0F566A3E0F567A3E0F568A32F
:10015600E0F56912186B7564FF75650F75660C75A9
:1001660067FF75680F7569187BFF7A0E79E51218B7
:100176006B7BFF7A0F792112186B7BFF7A0F7987D9
:1001860012186B7BFF7A0F79B4906347E0F564A38E
:10019600E0F565A3E0F566A3E0F56712186B7BFF53
:1001A6007A0F79DE906350E0F564A3E0F565A3E08D
:1001B600F566A3E0F56712186B7BFF7A10790C9051
:1001C6006354E0F564A3E0F565A3E0F566A3E0F506
:1001D6006712186B7BFF7A10793A90633DE0F564FD
:1001E600A3E0F565A3E0F566A3E0F56712186B7B5F
:1001F600FF7A10795D906339E0F564A3E0F565A3B5
:10020600E0F566A3E0F56712186B7BFF7A10797A42
:10021600906358E0F56412186B7BFF7A1079A4128C
:10022600186B7BFF7A1079CDA20EE433F5641218B1
:100236006B7BFF7A1079FD906683E0F56412186B8C
:100246007BFF7A11792A90668DE0F56412186B7B34
:10025600FF7A11795D9062B6E0F56412186B7BFF48
:100266007A11798BA201E433F56412186B7BFF7A5D
:100276001179B790667DE0F564A3E0F565A3E0F536
:1002860066A3E0F567A3E0F568A3E0F56912186BCD
:10029600122A747BFF7A12790212186B2290637805
:1002A600E0644C70527E127F08122E7D906380E0CF
:1002B600F55BA3E0F55CE4F55D7D03AF5CAE5B1238
:1002C6002F5E7E127F43122E7DAE5BAF5CE4FB7D1C
:1002D600101230387E127F46122E7D7410255CF582
:1002E6005CE4355BF55B055DE55DC3941040CA7E55
:1002F600127F46122E7D22906378E0646C705CF566
:100306005F7E127F48122E7DE4F55EAF5F7E007D34
:1003160003122F5E7E127F43122E7DE4F55DA85FE9
:10032600E6FF7482255DF582E43463F583EFF0051C
:100336005F055DE55DB410E67E637F82E4FB7D10BC
:100346001230387E127F46122E7D055EE55EC3941E
:100356000840B87E127F46122E7D22906378E064B4
:100366004B7061F55D746A255DF582E43463F5834F
:10037600E06032746A255DF582E43463F583E0F467
:100386006023746A255DF582E43463F583E0FF74C7
:1003960080255DF582E43463F583E0B50710055DDD
:1003A600E55DB408C09061047432F002085F9063A2
:1003B600787421F0300A0302085F7E127F83122EC2
:1003C6007D02085F906378E0B4521A200A077E1215
:1003D6007F8B122E7D9063787472F07E637F787DBA
:1003E6000812351122906378E064497045200A07A7
:1003F6007E127F96122E7D906380E0F55BA3E0F57A
:100406005CE4F55D855C82855B83E0FF7482255D37
:10041600F582E43463F583EFF0055CE55C70020574
:100426005B055DE55DB480DC7E637F787D8A123591
:100436001122906378E064437079A3E064527046B9
:10044600200A077E127F9E122E7D906380E0F55B68
:10045600A3E0F55CE4F55D855C82855B83E493FF50
:100466007482255DF582E43463F583EFF0055CE57F
:100476005C7002055B055DE55DB480DB7E637F78BD
:100486007D8A12351122906379E064576003020871
:1004960068906380E0F55BA3E0F55C7482255DF50A
:1004A60082E43463AD82FC7B80AF5CAE5B123BB210
:1004B60002085F906378E06444600302054A906333
:1004C60080E0FF6444700302085FEFB4310CC20A97
:1004D6007E127FA7122E7D02085F906380E0B43003
:1004E6000CD20A7E127FB3122E7D02085F906380C3
:1004F600E0B4320CD20B7E127FC0122E7D02085F52
:10050600906380E0B4330CC20B7E127FCE122E7D38
:1005160002085F906380E0B4340CD20C7E127FDD5B
:10052600122E7D02085F906380E0B4350CC20C7E0B
:10053600127FEA122E7D02085F906380E0FF123C74
:10054600BF02085F906104E07013200A077E127FE5
:10055600F8122E7D9063787421F002085F90610492
:100566007432F0906378E0FFB45104C2AF80FEEFBE
:1005760064577045200A077E137F06122E7D90630E
:1005860081E0906334F0E4F55D906334E0FFE55D6F
:10059600C39F400302085F7482255DF582E43463DD
:1005A600F583E0FF906380E0255D24AFF582E434B7
:1005B60061F583EFF0055D80D0906378E064536069
:1005C6000302066D200A077E137F11122E7D9063AB
:1005D60041E0FF9061B8E06F703C906342E0FF90AD
:1005E60061B9E06F7030906343E0FF9061BAE0B5A7
:1005F6000724906344E0FF9061BBE0B50718906361
:1006060045E0FF9061BCE0B5070C906346E0FF90C3
:1006160061BDE06F60169063787421F0300A0302C2
:10062600085F7E137F20122E7D02085FE4F55DE4ED
:10063600F50DAF5DFE74AF255DF582E43461F5839B
:10064600E0FD123C81055DE55DC394FE40E1C2AF6D
:10065600E4907FF0F0A3F0907FFD74AAF0A374FFFE
:10066600F0A37455F080FE906378E0644F704C9070
:100676006380E0F55BA3E0F55CE55C455B700A2012
:100686000A077E137F29122E7D200A077E137F30EC
:10069600122E7DE4F55D7482255DF582E43463F502
:1006A60083E0855C82855B83F0055CE55C70020512
:1006B6005B055DE55DB480DE02085F906378E0FF70
:1006C600B44521906380E0FDA3E0907FF0CDF0A3D8
:1006D600EDF0C2AF907FFD74AAF0A374FFF0A3748F
:1006E60055F080FEEF6465600302085F906380E06A
:1006F600FFA3E0907FF0CFF0A3EFF0E4F55BF55CAD
:10070600D3907FF1E0955C907FF0E0955B4020E42C
:10071600F50D255CFFE55B3401FE855C82855B8318
:10072600E0FD123C81055CE55C7002055B80D17ED4
:10073600137F32123408EF4E602012000390634795
:10074600EFF0120003906348EFF012000390634944
:10075600EFF012000390634AEFF07E137F381234F5
:1007660008EF4E6020120003906350EFF012000372
:10077600906351EFF0120003906352EFF012000302
:10078600906353EFF07E137F3E123408EF4E6020E5
:10079600120003906354EFF0120003906355EFF0DC
:1007A600120003906356EFF0120003906357EFF0C8
:1007B6007E137F44123408EF4E60201200039063CC
:1007C6003DEFF012000390633EEFF01200039063DA
:1007D6003FEFF0120003906340EFF07E137F4A1262
:1007E6003408EF4E6020120003906339EFF01200D8
:1007F6000390633AEFF012000390633BEFF01200B0
:100806000390633CEFF07E137F50123408EF4E6086
:10081600081239A4906358EFF0E4F55DE4F50DE5B0
:100826005D2401FFE433FE7439255DF582E434630B
:10083600F583E0FD123C81055DE55DC3944340DC34
:10084600C2AFE4907FF0F0A3F0907FFD74AAF0A30E
:1008560074FFF0A37455F080FE7E637F787D0812E6
:0208660035114A
:01086800226D
:103B7A00AE07EEC39430400BEED394395005EE24D1
:103B8A00D0FF22EEC39461400BEED394665005EE4B
:103B9A0024A9FF22EEC39441400BEED3944650056C
:083BAA00EE24C9FF22AF062240
:103C67009062AFE004F070069062AEE004F09062FC
:0A3C7700AEE0FEA3E0FF123C4B227A
:10000300123C67123B7AEFC454F0FEC006123C6701
:08001300123B7AD0E02FFF221E
:1039A400E4906A6EF0123C67906A6FEFF0C3943053
:1039B4004018E0FFD394395011906A6EE02407F563
:1039C40082E43461F583EFF08011906A6EE024079D
:1039D400F582E43461F583E4F0800C906A6EE004CF
:1039E400F0E0D3940840BE7563007564007565000B
:0C39F400E4F5667B017A61790712245328
:013A000022A3
:043408008E608F61E2
:10340C009062AEE4F0A374FFF0123C67EF606EF4D0
:10341C00606B856182856083E493B507EC7562010E
:10342C00E5612562F582E43560F583E493602590CF
:10343C0062AFE02562FF9062AEE03400FE123C4BBE
:10344C00E5612562F582E43560F583E493B5070404
:10345C00056280CCE5612562F582E43560F583E494
:10346C009370A6E56224FFFFE434FFFE9062AFE0A8
:10347C002FF09062AEE03EF07E007F0122E4FEFF72
:01348C00221D
:102D97007E137F81123408EF4E70037F01227E136A
:102DA7007F84123408EF4E600C123C67EF24D02466
:102DB700FF920E8002D20E7E137F8A123408EF4EE6
:102DC700600C123C67EF24D0906683F08005E49096
:102DD7006683F07E137F90123408EF4E600C123C2E
:102DE70067EF24D090668DF08005E490668DF07EC5
:102DF700137F96123408EF4E600C123C67EF24D015
:102E07009062B6F08005E49062B6F07E137F9C1264
:102E17003408EF4E600C123C67EF24D024FF920178
:102E27008002C20190634163A20190667D63A201A3
:102E37007F0612237C30013B7E137FA2123408EFFA
:102E47004E603012000390667DEFF012000390662B
:102E57007EEFF012000390667FEFF012000390669A
:102E670080EFF0120003906681EFF0120003906686
:062E770082EFF07F002253
:1020AE00C201E490668DF0D20EC204906683F09069
:1020BE0062B6F090634163A20190667D63A2017FD8
:1020CE000612237CE4F55BE55B75F003A424A8F50A
:1020DE0082E43413F583E493FB740193FA74029350
:1020EE00F9121E3D70030222A0E4F55CF55DFD744D
:1020FE002F2DF582E43461F583E0FF700302229BFD
:10210E00E55B75F003A424A8F582E43413F583E4AB
:10211E0093FB740193FA740293F9855C82758300C4
:10212E00121E56FEEFB50608755D01055C0222977C
:10213E00E55D7003022297EE6003022292E55B24B6
:10214E00FE602814700302227A14700302227E1499
:10215E00700302228614700302228A240560030291
:10216E00229B90668D7401F002229BD201742F2D5A
:10217E00F582E43461F583E0FF642D700302229B47
:10218E00123B7AEFC454F0FC74302DF582E43461C6
:10219E00F583E0FF123B7AEF2C90667DF074312DC3
:1021AE00F582E43461F583E0FF123B7AEFC454F01C
:1021BE00FC74322DF582E43461F583E0FF123B7A34
:1021CE00EF2C90667EF074332DF582E43461F58346
:1021DE00E0FF123B7AEFC454F0FC74342DF582E428
:1021EE003461F583E0FF123B7AEF2C90667FF0743A
:1021FE00352DF582E43461F583E0FF123B7AEFC4AE
:10220E0054F0FC74362DF582E43461F583E0FF1250
:10221E003B7AEF2C906680F074372DF582E43461B2
:10222E00F583E0FF123B7AEFC454F0FC74382DF5C1
:10223E0082E43461F583E0FF123B7AEF2C906681E5
:10224E00F074392DF582E43461F583E0FF123B7AA8
:10225E00EFC454F0FC743A2DF582E43461F583E05A
:10226E00FF123B7AEF2C906682F08021D204801D03
:10227E009066837401F08015C20E80119062B67460
:10228E0001F08009E4F55DF55C0D0220FD055B02B1
:02229E0020D549
:0122A000221B
:103AB000906579E0C3947C503D906579E0FE04F018
:103AC00074B72EF582E43462F583EFF0BF0A2790D5
:103AD0006579E0FF04F074B72FF582E43462F58372
:103AE000E4F0906579E0FF1235939065797408F001
:073AF0009062B8E004F0222F
:103A01009080007480F090633963A201F583F582A0
:103A110063A2017F0812237C90634163A20190801D
:103A21008863A2017F0A12237C908092E4F0A37440
:103A310032F0A37401F090634BE0FF9080B1F090FD
:103A410080E1EFF09080957455F0A3F090800074C0
:093A510001F09080097470F0226C
:10370A00908009E04410F09080A0E0706C9080A155
:10371A007482F09080A874FFF0A3F0A3F0A3F07F66
:10372A00039080AEEFF07FCBA3EFF07F039080ACE5
:10373A00EFF0A374CBF09080007402F0906A6212EA
:10374A001F7C00000000906A62E0908040F0906A5E
:10375A0063E0908041F0906A64E0908042F0906A61
:10376A0065E0908043F0A3E4F0A3F0A3F0A3F09007
:09377A008018F0A3F0A3F0A3F005
:013783002223
:1038E100908009E04440F09080D17482F090634C64
:1038F100E0FF9080DEF090634DE0FF9080DFF0907C
:1039010080027402F0906A66121F7C000000009031
:103911006A66E0908058F0906A67E0908059F09074
:103921006A68E090805AF0906A69E090805BF0A349
:10393100E4F0A3F0A3F0A3F0908030F0A3F0A3F0A3
:02394100A3F0F1
:013943002261
:10378400908009E04420F09080B8E0706C9080B99B
:103794007482F07F039080C6EFF07FCDA3EFF07FBB
:1037A400039080C4EFF0A374CDF09080C074FFF058
:1037B400A3F0A3F0A3F09080017402F0906A6A125F
:1037C4001F7C00000000906A66E090804CF0906AD4
:1037D40067E090804DF0906A68E090804EF0906AC7
:1037E40069E090804FF0A3E4F0A3F0A3F0A3F0907D
:0937F4008024F0A3F0A3F0A3F07F
:0137FD0022A9
:10348D008C5B8D5CA907EAFDE975F018A424ACFFEF
:10349D00E5F034808F82F583EDF0EBFDE975F018E2
:1034AD00A4FFAEF024ACFBEE34808B82F583A3ED4C
:1034BD00F0855C828C83E0FDEF24A8FFEE3480FE66
:1034CD008F82F583EDF0855C828C83A3E08F828EF5
:1034DD0083A3F0855C82855B83A3A3E0FDE975F092
:1034ED0018A424A8FFE5F03480FE8F82F583A3A3F2
:1034FD00EDF0855C828C83A3A3A3E08F828E83A3E2
:04350D00A3A3F02262
:063511008D60AB07AA0665
:10351700906A62E0FCA3E0FDA3E0FEA3E0F5648E01
:10352700638D628C61AE02AF038E838F8263A201CB
:10353700E563540744C0F58385648263A201AF60E5
:103547001223E5908000E020E5F9E4FCFDFEE56448
:103557002560F564EE3563F563ED3562F562EC35AC
:1035670061F561908040E561F0A3E562F0A3E56352
:10357700F0A3E564F09080007420F0AF64AE63AD13
:0B35870062AC61906A62121F70AF60BE
:013592002216
:06368F008D5BAB07AA06EB
:10369500906A66E0FCA3E0FDA3E0FEA3E0F55F8E83
:1036A5005E8D5D8C5CAE02AF038E838F8263A2015B
:1036B500E55E540744D0F583855F8263A201AF5B65
:1036C5001223E5E4FCFDFEE55F255BF55FEE355E67
:1036D500F55EED355DF55DEC355CF55C908058E5A6
:1036E5005CF0A3E55DF0A3E55EF0A3E55FF09080F7
:1036F500027420F0AF5FAE5EAD5DAC5C906A6612A1
:043705001F70AF5B27
:01370900229D
:02310C008F5BD7
:10310E00908001E030E5037F0022906A6AE0FCA324
:10311E00E0FDA3E0FEA3E0F55F8E5E8D5D8C5C901E
:10312E00667D63A201E55E540744C8F583855F8220
:10313E0063A2017F061223FBE55F2406F55FE435EB
:10314E005EF55EE4355DF55DE4355CF55C90657BC2
:10315E0063A201E55E540744C8F583855F8263A2CE
:10316E0001AF5B1223FBE4FCFDFEE55F255BF55F23
:10317E00EE355EF55EED355DF55DEC355CF55C903E
:10318E00804CE55CF0A3E55DF0A3E55EF0A3E55FA2
:10319E00F09080017420F0AF5FAE5EAD5DAC5C90E0
:0731AE006A6A121F70AF5B9B
:0131B50022F7
:102C93009081E0E0F55B055B055B055B055B055B30
:102CA300055B055B055B055B055B908010E0F55EEE
:102CB300A3E0F55FA3E0F560A3E0F5619081E1E0B7
:102CC300F55B055B055B055B055B055B055B055B11
:102CD300055B055B055B908014E0F562A3E0F5639B
:102CE300A3E0F564A3E0F565E564B56008E565B5C3
:102CF30061037F0022E4F55BE564540744E0F58358
:102D030085658263A20190637863A2017F08122420
:102D13001390637A63A2019062B063A2017F0612EB
:102D2300237C906378E0F55CA3E0F55DE4F55B90CC
:102D33006378E0702AA3E024F8F55BE56454074464
:102D4300E0F58385658274082582F582E43583F591
:102D53008363A20190637863A201AF5B122413AE75
:102D63005CE4FCFDE565255DF565E5643EF564ED34
:102D73003563F563EC3562F562908014E562F0A388
:102D8300E563F0A3E564F0A3E565F090800074408B
:032D9300F0AF5B43
:012D9600221A
:102799009081E6E0F55B055B055B055B055B055B29
:1027A900055B055B055B055B055B908028E0F55ED5
:1027B900A3E0F55FA3E0F560A3E0F5619081E7E0B0
:1027C900F55B055B055B055B055B055B055B055B10
:1027D900055B055B055B90802CE0F562A3E0F56382
:1027E900A3E0F564A3E0F565E4F55BE564B5600A8B
:1027F900E565B56105C2080228F3E564540744F0AC
:10280900F58385658263A20190637863A2017F08DD
:10281900122413906378E0F55CA3E0F55DE55D456E
:102829005C70099080027410F07F0022906684E049
:10283900FFF4602D90637AE06F7076906685E0FF13
:1028490090637BE06F706A906686E0FF90637CE03E
:102859006F705E906687E0FF90637DE06F60228015
:102869005090637AE0906684F090637BE09066858F
:10287900F090637CE0906686F090637DE0906687D7
:10288900F0906378E0702AA3E024F8F55BE56454DE
:102899000744F0F58385658274082582F582E4355D
:1028A90083F58363A20190637863A201AF5B12246D
:1028B90013AE5CE4FCFDE565255DF565E5643EF573
:1028C90064ED3563F563EC3562F562AF61AE60AD19
:1028D9005FAC5EAB65AA64A963A862D3121F5F40AF
:1028E900099080027410F07F002290802CE562F03C
:1028F900A3E563F0A3E564F0A3E565F090800274B5
:0429090040F0AF5B90
:01290D0022A7
:10290E009081E3E0F55B055B055B055B055B055BB5
:10291E00055B055B055B055B055B90801CE0F55E6A
:10292E00A3E0F55FA3E0F560A3E0F5619081E4E03C
:10293E00F55B055B055B055B055B055B055B055B99
:10294E00055B055B055B908020E0F562A3E0F56317
:10295E00A3E0F564A3E0F565E4F55BE564B5600A14
:10296E00E565B56105C209022A59E564540744E8D4
:10297E00F58385658263A20190600463A2017F0ED8
:10298E00122429906004E0F55CA3E0F55D90600CE4
:10299E00E0FFF4604590667DE0FEEF6E706EA3E0A2
:1029AE00FF90600DE06F706490667FE0FF90600EA8
:1029BE00E06F7058906680E0FF90600FE06F704C93
:1029CE00906681E0FF906010E06F7040906682E04C
:1029DE00FF906011E06F60048032D28D906004E051
:1029EE00702AA3E024F2F55BE564540744E8F5830E
:1029FE00856582740E2582F582E43583F58363A2A4
:102A0E000190600463A201AF5B122429AE5CE4FC6A
:102A1E00FDE565255DF565E5643EF564ED3563F52B
:102A2E0063EC3562F562AF61AE60AD5FAC5EAB6517
:102A3E00AA64A963A862D3121F5F5006E55D455CC8
:102A4E0070099080017410F07F0022908020E56262
:102A5E00F0A3E563F0A3E564F0A3E565F0908001D3
:052A6E007440F0AF5BB5
:012A73002240
:042E7D008E608F6173
:102E8100906A62E0FCA3E0FDA3E0FEA3E0F5678E9B
:102E9100668D658C64E567FFE5665407FEE42FF5F2
:102EA10063EE34C0F562856382F5837423F00563B4
:102EB100E563700205625362C7F582856283740A15
:102EC100F00563E563700205625362C79063416375
:102ED100A20185628385638263A2017F061223E5D5
:102EE10074062563F563E43562F562856083856167
:102EF1008263A20185628385638263A2011223C971
:102F0100908000E020E5F9E4FCFDFE906A62E0F8C3
:102F1100A3E0F9A3E0FAA3E02FFFEE3AFEED39FDBD
:102F2100EC38FCEF2408FFE43EFEE43DFDE43CFC0C
:102F3100906A62121F70906A62E0908040F0906A1D
:102F410063E0908041F0906A64E0908042F0906A82
:0C2F510065E0908043F09080007420F058
:012F5D002251
:063038008E608F618D62C5
:10303E00906A62E0FCA3E0FDA3E0FEA3E0F5688EDB
:10304E00678D668C65E568FFE5675407FEE42FF52E
:10305E0064EE34C0F563856482F5837423F00564F1
:10306E00E564700205635363C7F582856383EBF0F5
:10307E000564E564700205635363C790634163A200
:10308E000185638385648263A2017F061223E57442
:10309E00062564F564E43563F56385608385618296
:1030AE0063A20185638385648263A201AF621223EA
:1030BE00E5908000E020E5F974082562F562FFE4F2
:1030CE00FCFDFEE5682FF568EE3567F567ED3566B4
:1030DE00F566EC3565F565908040E565F0A3E5662F
:1030EE00F0A3E567F0A3E568F09080007420F0AFE0
:0D30FE0068AE67AD66AC65906A62121F7027
:01310B0022A1
:023593008F7532
:10359500906A62E0FCA3E0FDA3E0FEA3E0F5798E6E
:1035A500788D778C76E579FFE5785407FEE42FFF73
:1035B500EE34C09062B763A201F5838F8263A201E6
:1035C500AF751223E5908000E020E5F9E4FCFDFEEF
:1035D500E5792575F579EE3578F578ED3577F57773
:1035E500EC3576F576908040E576F0A3E577F0A3A7
:1035F500E578F0A3E579F09080007420F0AF79AE1E
:0B36050078AD77AC76906A62121F70FF
:013610002297
:062F5E008E608F61AB05DF
:102F6400906A62E0FCA3E0FDA3E0FEA3E0F5678EB7
:102F7400668D658C64E567FFE5665407FEE42FF50E
:102F840063EE34C0F562856382F5837423F00563D0
:102F9400E563700205625362C7F582856283EBF0D4
:102FA4000563E5637002056290634163A201856273
:102FB4008385638263A2017F061223E57406256379
:102FC400F563E43562F5625362C7E5608563828523
:102FD4006283F00563E563700205625362C7F5829C
:102FE400856283E561F00563E563700205625362FF
:102FF400C7908000E020E5F9E567240AF567E43529
:1030040066F566E43565F565E43564F564908040FD
:10301400E564F0A3E565F0A3E566F0A3E567F09049
:1030240080007420F0AF67AE66AD65AC64906A62F0
:03303400121F70F8
:013037002276
:103C4B00E5D220E0FBC2AF438E2075D2028F828E6D
:0B3C5B0083E0FFE4F5D2538EDFD2AF10
:013C6600223B
:103C8100E5D220E0FBC2AF43D2028F828E83EDF0FA
:093C910075D25063D250D2AF226B
:10361100E4FDED2401FFE433FE123C4B74392DF53A
:1036210082E43463F583EFF00DBD3FE6E4FDED2464
:103631007FFFE433FE123C4B742F2DF582E434619D
:10364100F583EFF0742F2DF582E43461F583E0709A
:103651001B742F2DF582E43461F5837420F07430EE
:103661002DF582E43461F583E4F080040DBD80BE64
:10367100E49061AEF0FDEDFF7E00123C4B74AF2D86
:0D368100F582E43461F583EFF00DBDFEE944
:01368E002219
:023BB2008B6026
:103BB400A2AF920FC2AF85A26153A2FE8E838F8201
:103BC40005A28C838D827409122441E56053A2FE00
:103BD40043A22012244353A2DF8561A2A20F92AF15
:013BE400FFE1
:013BE50022BD
:103C2E00A2AF920FC2AF8C838D82EF12244143A2BA
:0C3C3E002012244353A2DFA20F92AFFF1C
:013C4A002257
:023BE6008F5BF3
:103BE800A2AF920FC2AFE4F5838D8274061224410E
:103BF800E55B43A22012244353A2DFA20F92AF7FBA
:013C080001BA
:013C09002298
:023C0A008F5BCE
:103C0C00A2AF920FC2AFE4F5838D82740A122441E5
:103C1C00E55B43A22012244353A2DFA20F92AF7F95
:013C2C000196
:013C2D002274
:1022A100A907E7FFA805EF93C3966008403B74FCBC
:1022B1002FFF80F00F08EF93C3966008402B74FB4B
:1022C1002FFF80E00F08EF93C3966008401B74FA5C
:1022D1002FFF80D00F08EF93D3966008400B74F95D
:1022E1002FFF80C01F1F1F1F1FEF54FEF80303F7AE
:1022F100E893FC08E893FD08E893FE08E893FF22C1
:1023010009E993C39D6008402974FB29F980F1090B
:10231100E993C39E6008401A74FA29F980E209E939
:1023210093D39F6008400B74F929F980D3191919C7
:102331001919E9C313C313FF22740093F8ECC3986E
:102341004024701F740193F8EDC398401970147400
:0E2351000293F8EEC398400E7009740393F8DF
:10235F00EFC39840037F00227F0122EDF8E6F008DB
:10236F00A3DFFA22EDF8E0F608A3DFFA22E0A36379
:10237F00A201F0A363A201DFF475A20022E0A36320
:10238F00A201F0A363A201E0A363A201F0A363A2E1
:10239F0001E463A201F0A363A201DFE175A20022B1
:1023AF00E0A363A2016DFE936CFDEE058393FC1514
:1023BF008363A201DFEA75A200227F00E493A36387
:1023CF00A201F00F600CA3E583C2E3F58363A201C2
:1023DF0080EA75A20022E0A363A201F0A3E583C205
:1023EF00E3F58363A201DFEE75A20022E0A363A2EF
:1023FF0001F0A3E583C2E4D2E3F58363A201DFEC2E
:10240F0075A20022E583C2E3F583E0A363A201F086
:10241F00A363A201DFEE75A20022E583C2E4D2E33B
:10242F00F583E0A363A201F0A363A201DFEC75A221
:10243F000022F922C002C004C00612FFF0D006D05D
:04244F0004D0022291
:1013C0003C6D303D003C6D313D003C6D323D003C9C
:1013D0006D333D003C6D343D003C6D353D003C6D52
:1013E000363D003C6D373D003C6D383D003C6D396D
:1013F0003D003C6D31303D003C6D31313D003C6D78
:1014000031323D003C6D31333D003C6D31343D00A7
:101410003C6D31353D003E2A2C312CCFE0F0E0EC24
:10142000E5F2F0FB20F8E8EDFB2043414E0A003ED8
:101430004C2C6B30312C25732C43EAEEF0EEF1F29C
:10144000FC20EDE020F8E8EDE52043414E2C302073
:101450002D20353030EAE1283530EC292C31202D93
:10146000203530EAE128353030EC290A0030202DD3
:1014700020353030EAE1283530EC290031202D20AC
:101480003530EAE128353030EC29003E2A2C312C69
:10149000CFE0F0E0ECE5F2F0FB20EFF0EEF2EEEA68
:1014A000EEEBE0204D4F444255530A003E4C2C4990
:1014B00030312C256C752CD1EAEEF0EEF1F2FC20E7
:1014C000EEE1ECE5EDE02C35302C3130302C3330D2
:1014D000302C3630302C313230302C323430302C0D
:1014E000343830302C393630302C31393230302CE1
:1014F00033383430302C35373630302C31313532CA
:1015000030300A003E532C4931322C2562752CC0F4
:10151000E4F0E5F120E1EBEEEAE020D2C8D220EDE4
:10152000E020F8E8EDE50A003E422C4930322C2557
:1015300062752CC2FBF1F2E0E2EBFFF2FC205254A8
:101540005320EFF0E820EFE5F0E5E4E0F7E50A00EE
:101550003E532C6D2562752C2562752D25752D2524
:1015600062752D2562752CCFF0E8E1EEF020256242
:10157000752028B9CFF02DD0E5E32DCAEEEB2DD2A2
:10158000E8EF290A003E532C5630382C2562752C82
:10159000C8EDF2E5F0E2E0EB20EEEFF0EEF1E0284E
:1015A0002A3130ECF1290A003C21003C6B30313DFE
:1015B000003C4930313D003C4930323D003C49312E
:1015C000323D003C5630383D002043616E45724745
:1015D000495400200A002043616E4572724348213D
:1015E000000A000AC7E0EFF0EEF10A00CEF8E8E1E9
:1015F000EAE020CAD1210A00CFF0E8EDFFF2EE3A8E
:1016000000CED8C8C1CAC0210000C1814001C0803D
:101610004101C0804100C1814001C0804100C181C1
:101620004000C1814001C0804101C0804100C181B2
:101630004000C1814001C0804100C1814001C080A3
:101640004101C0804100C1814001C0804100C18191
:101650004000C1814001C0804100C1814001C08083
:101660004101C0804100C1814000C1814001C08072
:101670004101C0804100C1814001C0804100C18161
:101680004000C1814001C0804101C0804100C18152
:101690004000C1814001C0804100C1814001C08043
:1016A0004101C0804100C1814000C1814001C08032
:1016B0004101C0804100C1814001C0804100C18121
:1016C0004000C1814001C0804100C1814001C08013
:1016D0004101C0804100C1814001C0804100C18101
:1016E0004000C1814001C0804101C0804100C181F2
:1016F0004000C1814001C0804100C1814001C080E3
:101700004101C0804100C1814000C0C101C303024A
:10171000C2C60607C705C5C404CC0C0DCD0FCFCE7D
:101720000E0ACACB0BC90908C8D81819D91BDBDAAD
:101730001A1EDEDF1FDD1D1CDC14D4D515D71716CD
:10174000D6D21213D311D1D010F03031F133F3F2DD
:101750003236F6F737F53534F43CFCFD3DFF3F3EBD
:10176000FEFA3A3BFB39F9F83828E8E929EB2B2A4D
:10177000EAEE2E2FEF2DEDEC2CE42425E527E7E60D
:101780002622E2E323E12120E0A06061A163A3A27D
:101790006266A6A767A56564A46CACAD6DAF6F6EFD
:1017A000AEAA6A6BAB69A9A86878B8B979BB7B7A2D
:1017B000BABE7E7FBF7DBDBC7CB47475B577B7B64D
:1017C0007672B2B373B17170B0509091519353521D
:1017D0009296565797559594549C5C5D9D5F9F9E3D
:1017E0005E5A9A9B5B99595898884849894B8B8ACD
:1017F0004A4E8E8F4F8D4D4C8C448485458747468D
:091800008682424383418180404D
:103B410052668F000000000000000000000000002D
:103B5100000000000020203A13C013C513CA13CF80
:103B610013D413D913DE13E313E813ED13F213F88F
:083B710013FE1404140A1410E1
:013CBF0022E2
:03002300023A5A44
:103A5A00C0E0C083C082C0D075D018309817750BEB
:103A6A0001D291743D2536F582E43469F583E599EE
:103A7A00F00536C298309925E538C395355013AF0D
:103A8A00380538743D2FF582E4346AF583E0F599F8
:103A9A008009AF358F38EF60020538C299D0D0D08F
:063AAA0082D083D0E0325F
:102A74007BFF7A14791612186B9068A1E0701475B4
:102A840064FF75651475666D7BFF7A14792F1218CF
:102A94006B80127564FF75651475667C7BFF7A1410
:102AA400792F12186B7BFF7A14798B12186B906A4A
:102AB40060E0FEA3E0FFC3E49FFFE49EFEAB07FAE1
:102AC4003395E0F9F87F007E8C7D0A7C00121EBFEE
:102AD4008F678E668D658C647BFF7A1479AC1218CF
:102AE4006B7BFF7A1579049068A2E0F56412186B89
:102AF4007BFF7A157928A21AE433F56412186BE483
:102B0400F5607BFF7A157950856064E560FD339547
:102B1400E0FC74A72DF58274683CF583E0F565AF9D
:102B240060EF3395E0FEEF25E0FFEE33FE74BA2F3D
:102B3400F58274683EF583E0F566A3E0F56774DA20
:102B44002DF58274683CF583E0F568AF60EF33954A
:102B5400E0FE74EC2FF58274683EF583E0F569E5D8
:102B64006004F56A12186B0560C3E5606480949094
:102B740040907BFF7A157985906A5FE0F5641218BE
:012B84006BE5
:012B8500222D
:1025F7007E157FA8123408EF4E70037F0122E49006
:1026070068A1F07E157FAB123408EF4E601B123CB9
:10261700678F5BE55BB431069068A1740AF0E55BF0
:10262700B432069068A17464F07E157FB112340845
:10263700EF4E60231239A4A804A905AA06AB077FA9
:10264700007E8C7D0A7C00121EBF121F51906A60AB
:10265700EEF0A3EFF0800A906A6074FFF0A374B8FD
:10266700F07E157FB7123408EF4E600C123C67EF0F
:1026770024D024FF921A8002C21A7E157FBD12341D
:1026870008EF4E600A1239A49068A2EFF08005E4C3
:102697009068A2F07E157FC3123408EF4E600D12CA
:1026A70039A4906A5EEEF0A3EFF08009906A5EE4C9
:1026B700F0A37464F0E4F55BE55B25E0243AF8E603
:1026C700FE08E6FF123408EF4E60681239A4E55B96
:1026D700FD3395E0FC74A72DF58274683CF583EF14
:1026E700F01239A4AD07AC06AF5BEF3395E0FEEF10
:1026F70025E0FFEE33FE74BA2FF58274683EF5834A
:10270700ECF0A3EDF01239A4E55BFD3395E0FC7422
:10271700DA2DF58274683CF583EFF01239A4E55B96
:10272700FD3395E0FC74EC2DF58274683CF583EF7E
:10273700F0804EE55BFD3395E0FC74A72DF58274C0
:10274700683CF583E4F0AF5BEF3395E0FEEF25E0FF
:10275700FFEE33FE74BA2FF58274683EF583E4F01A
:10276700A3F074DA2DF58274683CF583E4F0AF5B6F
:10277700EF3395E0FE74EC2FF58274683EF583E441
:10278700F0055BC3E55B6480949050030226BF7F2E
:012797000041
:01279800221E
:1038780043AB01C2E8C2EAE4FFEFC454F0F5B1C3B8
:10388800EF64809488500575B3D08003E4F5B3E401
:10389800F5B275BCC8F5BDF5BE75BF7875C4FFF542
:1038A800C5F5C675C778F5A3F5A3F5A3F5A3F5A3E4
:1038B800F5A3F5A3F5A30FBF0EBF9068A1E0FF2500
:1038C800E0F5B475B50C75B66C75A11275AB0275DB
:0838D800C13E75C3FF75C20378
:0138E00022C5
:1039440075B180E4F5B3F5B28525BCE5265403FFD3
:1039540033333354F8FFE52654E04FFFE527C4130F
:1039640054074FF5BDE52733333354F8FFE528C436
:103974001354074FF5BEE52833333354F8F5BF85A8
:103984002AA3852BA3852CA3852DA3852EA3852F60
:10399400A38530A38531A3E529540F2450F5B32220
:102B8600E59B541F6020200A1A7E157FC9122E7DF0
:102B9600E59B541FFF7E007D03122F5E7E157FD3BB
:102BA600122E7DE4F59BE5BA30E008E4F5B375B185
:102BB60080F5B2E5CFF47003022C90755D01E4F563
:102BC6005CE5CFF4555D7003022C7EE55CC454F0E1
:102BD600F5B1E5B2547F6420706FE5B3540FF52963
:102BE60085BC25E5BD541FFF131313541FFFE5BD18
:102BF60054E044184FF526E5BDC43354E0FFE5BE66
:102C0600131313541F4FF527E5BEC43354E0FFE5F5
:102C1600BF131313541F4FF52885A32A85A32B85AD
:102C2600A32C85A32D85A32E85A32F85A33085A34D
:102C360031E4F5B2E525547EB5250575B35080031C
:102C460075B3D0E5292405FF22E5B2549F60232001
:102C56000A207E157FD6122E7DAFB27E007D03122E
:102C66002F5EAFB37E007D03122F5E7E157FE112CD
:102C76002E7DE4F5B275B3D0E55D25E0F55D055C26
:0C2C8600E55CC394085003022BC77F00DC
:012C9200221F
:1037FE00C219C21CE4F536F50BD296C21B753705FD
:10380E009068A5F0A3F0F534F535F538FF7F4090BC
:10381E0068FDE4F0A3DFFCE49068B8F0A3F09068D4
:10382E00EAF0906A5DF01225F7123878C2ADE4F531
:10383E00C9D2CDD2CCC2C9C2CAF5CDF5CC906A6080
:10384E00E0F5CBA3E0F5CA85CBCD85CACCE4F598DF
:10385E00D29E438740C29FC2ACC298C29975B8101F
:09386E0075B710D2CAD29CD2AC8D
:01387700222E
:013CC00022E1
:013CC10022E0
:05001E00D29CD2AC22CF
:033CBC00D21C22F5
:063AF700AC05AB07AA06B6
:103AFD009068EB74FFF09068FCF0AF041CEF602D44
:103B0D000BEBAE0270010A14F5828E83E0FF906814
:103B1D00EBE06FFF90160993FE9068FCE06E9068E5
:0D3B2D00EBF0EF901709939068FCF080CD4D
:013B3A002268
:1032EB00053474EC2534F582E43468F583E070081A
:1032FB00F5349068B8F0A3F074A72534F582E43464
:10330B0068F583E0906A3DF074EC2534F582E43483
:10331B0068F583E0906A3EF0E53425E024BAF58247
:10332B00E43468F583E0FCA3E0FDEC906A3FF0A386
:10333B00EDF0E4A3F074DA2534F582E43468F58318
:10334B00E0906A42F07E6A7F3D7D06123AF7906804
:10335B00EBE0906A43F09068FCE0906A44F0E4F58F
:10336B0038753508301A02C296C2992099FDD29948
:01337B00222F
:1031B600906A5DE0C394404002E4F0906A5DE024CA
:1031C600FDF582E43468F583E0FF30E179906A5DCD
:1031D600E0FE24FDF582E43468F583EF54FDF0E467
:1031E600906478F0A3740DF090667CE090647AF0B9
:1031F600A37419F0A37448F0A37479F0EE131313B3
:10320600541FFF9068A2E02F90647EF0906A5DE004
:10321600FD540725E025E0248090647FF0A3740820
:10322600F0F5F0EDA424A1F582E5F03466F58363AC
:10323600A20190648163A2017F0812237C906A5DDB
:0F324600E004F07F0122906A5DE004F07F002237
:013CC20022DF
:101B6500E538D39535401F906A5FE024FEFF906A03
:101B75005EE034FFFEC39068A6E09F9068A5E09EF6
:101B85005004D296C2909068EAE0C394404002E4C3
:101B9500F09068EAE024FDF582E43468F583E020FE
:101BA500E0069068EAE004F0122B86EF606FE52806
:101BB500640F70699068A2E0FF652770609068EA1D
:101BC500E024FDF582E43468F583E0FE30E04E90D4
:101BD50068EAE0FD24FDF582E43468F583EE54FE01
:101BE500F0752548752679ED131313541FFEEF2E56
:101BF500F5279068EAE0FF540725E025E02480F505
:101C05002875290875F008EFA424A1F582E5F034BC
:101C150066F5837D2A7F08122373123944300257F3
:101C25009068A6E004F070069068A5E004F0C20292
:101C35009068A4E004F070069068A3E004F0D390E7
:101C450068A4E094B89068A3E0940B402AE4F0A35C
:101C5500F0F55B74FD255BF582E43468F583E030CF
:101C6500E20E74FD255BF582E43468F5837403F0B8
:101C7500055BE55BB440DC906A5EE0FEA3E0FF2413
:101C8500FEFDEE34FFFC9068A5E0FAA3E0FBD39DD2
:101C9500EA9C4005309602C296D3EB9FEA9E40230C
:101CA500D2901232EBC291E49068A5F0A3F0200A1D
:101CB500127E157FE3122E7D7E6A7F3DE4FB7D0853
:101CC500123038E536D394005003021E3CE50BD3A1
:101CD50095375003021E3C906A5FE024FEFE906A31
:101CE5005EE034FF9068A5F0A3CEF0C29185363949
:101CF500E4F536F50B7E697F3D90693FE02405FDEF
:101D0500123AF79068FCE0FF9068EBE04F600A201C
:101D15000A077E157FEC122E7D200A127E157FF8AC
:101D2500122E7D7E697F3DE4FBAD3912303874A7F4
:101D35002534F582E43468F583E0FF90693DE0B52C
:101D4500071474EC2534F582E43468F583E0FF90DC
:101D5500693EE06F600A200A077E167F01122E7D1C
:101D6500E4F55B90693FE0FFE55BC39F4003021E1E
:101D75003C9068B8E0FEA3E0FF24A1F58274663EBE
:101D8500F583E0FD7441255BF582E43469F583E074
:101D9500FCED6C602274A12FF58274663EF583EC30
:101DA500F0EF7803CEC313CE13D8F924FDF5827472
:101DB500683EF5837403F09068B9E004F07006900E
:101DC50068B8E004F09068B8E0FCA3E0FDAE0478E4
:101DD50003CEC313CE13D8F9FF24FDF58274683EF4
:101DE500F583E04404F074A12DF58274663CF58317
:101DF500E0FD7440255BF582E43469F583E0FCED94
:101E05006C601F9068B8E0FAA3E024A1F5827466BF
:101E15003AF583ECF074FD2FF58274683EF5837412
:101E250003F09068B9E004F070069068B8E004F03B
:071E3500055B055B021D685F
:011E3C002283
:0B3CB100301C05C21C7F01227F002296
:10338800020869E493A3F8E493A34003F68001F2EA
:1033980008DFF48029E493A3F85407240CC8C33346
:1033A800C4540F4420C8834004F456800146F6DF15
:1033B800E4800B0102040810204080903B3BE47E2F
:1033C800019360BCA3FF543F30E509541FFEE4930A
:1033D800A360010ECF54C025E060A840B8E493A3D1
:1033E800FAE493A3F8E493A3C8C582C8CAC583CAFC
:1033F800F0A3C8C582C8CAC583CADFE9DEE780BEB4
:013B7900004B
:101E3D00BB010689828A83E0225002E722BBFE02A3
:091E4D00E32289828A83E49322D6
:101E5600BB010CE58229F582E5833AF583E0225041
:101E660006E92582F8E622BBFE06E92582F8E2228B
:0D1E7600E58229F582E5833AF583E49322A5
:101E830075F008758200EF2FFFEE33FECD33CDCC16
:101E930033CCC58233C5829BED9AEC99E582984099
:101EA3000CF582EE9BFEED9AFDEC99FC0FD5F0D676
:101EB300E4CEFBE4CDFAE4CCF9A88222B800C1B9A0
:101EC3000059BA002DEC8BF084CFCECDFCE5F0CBDE
:101ED300F97818EF2FFFEE33FEED33FDEC33FCEB17
:101EE30033FB10D703994004EB99FB0FD8E5E4F9D2
:101EF300FA227818EF2FFFEE33FEED33FDEC33FCBF
:101F0300C933C910D7059BE99A4007EC9BFCE99AB2
:101F1300F90FD8E0E4C9FAE4CCFB2275F010EF2FF7
:101F2300FFEE33FEED33FDCC33CCC833C810D707F7
:101F33009BEC9AE899400AED9BFDEC9AFCE899F832
:0E1F43000FD5F0DAE4CDFBE4CCFAE4C8F922C5
:0E1F5100C3E49FFFE49EFEE49DFDE49CFC22A1
:101F5F00EB9FF5F0EA9E42F0E99D42F0E89C45F0D8
:011F6F00224F
:0C1F7000ECF0A3EDF0A3EEF0A3EFF022E4
:101F7C00A8828583F0D083D082121F93121F9312F4
:101F8C001F93121F93E473E493A3C583C5F0C58319
:101F9C00C8C582C8F0A3C583C5F0C583C8C582C8AF
:011FAC002212
:10180900E5702464F8E60570227861301602786480
:10181900E475F00112200E021E3D200FEB7F2ED23F
:101829000F8018EF540F2490D43440D4FF30130B99
:10183900EF24BFB41A0050032461FFE5716002155B
:10184900710574E5747002057330160D7861E475DD
:10185900F00112200EEF021FAD023AB07403D21646
:101869008003E4C216F5708B618A628963E4F571BD
:10187900F573F574E57160077F2012184480F575DA
:1018890072FFC210C20FC211C212C214C215C2170E
:10189900121812FF700D3016057F00121855AF741B
:1018A900AE7322B4255FC2D5C213121812FF24D019
:1018B900B40A00501A75F00A787130D50508B6FFD8
:1018C9000106C6A426F620D5047002D21280D924B6
:1018D900CFB41A00EF5004C2E5D213021A55D21040
:1018E90080C6D20F80C0D21180BCD2D580BAD214A2
:1018F90080B47F201218442011077401B57100408B
:10190900F1121809FF12184402187DD217D2158056
:1019190095121809FB121809FA121809F94A4B709D
:101929000679267A1B7BFF20112EE571602A7E003D
:101939008E82758300121E5660060EEE657270F077
:10194900C2D5EBC0E0EAC0E0E9C0E0EE121A9CD0D3
:10195900E0F9D0E0FAD0E0FB121E3DFF60AAEBC02F
:10196900E0EAC0E0E9C0E0121844D0E02401F9D06F
:10197900E03400FAD0E0FBE5720460DCD572D9806E
:10198900877BFF7A1A7998D211809C791080027925
:1019990008C215C2178008D2D5790A8004790AC20B
:1019A900D5E572047002F572E4FAFDFEFF1218091A
:1019B900FC7B08201013121809FD7B10300F0A1246
:1019C9001809FE121809FF7B20EC3382D592D550F5
:1019D90013C3E4300F069FFFE49EFEE42010039D2D
:1019E900FDE49CFCE4CBF8C210EC700CCFCECDCC5E
:1019F900E824F8F870F38017C3EF33FFEE33FEEDF8
:101A090033FDEC33FCEB33FB994002FB0FD8E9EBD8
:101A1900301005F8D0E0C448B210C0E00AEC4D4ED1
:101A29004F78207B0070C2EAB5720040BCC0E0125A
:101A39001A9ED0F0D0E0201004C4C0E0C4B210C097
:101A4900F012182DD0F0D5F0EB02187D12206D1987
:101A59001A5319945818EB4C18E74219984F19A0C2
:0F1A69004419A04919004319A655198A46198A2C
:101A780045198A471B465018EF2D18F32E19162BB7
:101A880018F7231914201B2F2A18AF480000190E25
:101A98003F3F3F00790AA2D5201214301409B9102B
:101AA800020404B9080104A2D5201502500104203B
:101AB80011689211B571005034C0E07F20301219BE
:101AC8007F30A21172157214500F121AF5C211C28A
:101AD80015C214C2177F30800F301403E9C0E0121A
:101AE8001844301403D0E0F9D0E0B571CC301417A5
:101AF8007F30B9100C1218447F583013077F788054
:101B080003B908031218443011057F2D0218447FC9
:101B1800202017F87F2B2015F322921180CF286EF2
:101B2800756C6C2900D2101218093010F8C21078A0
:101B38007130D50108F60218AF2D504349581218D4
:101B4800092403B405004001E4901B4193121835A1
:0D1B5800743A121835D212757104021994F6
:102453008B608A618962E4F56CF56BF56AF569F561
:1024630067F568E564456545636012EBC0E0EAC063
:10247300E0E9C0E0AB63AA64A96512201EAB600566
:1024830062E562AA617002056114F9121E3DF56DE1
:10249300C394094007E56DD3940D40E1E56D6420D5
:1024A30060DBE56DB42D054368038016E56DB42B41
:1024B30005436801800C74FF2562F56274FF356182
:1024C300F561E56660046410703FAB60AA61A962C0
:1024D300121E3D64306009E566702E75660A802918
:1024E300900001121E56FF64786004EFB458134342
:1024F300680175661074022562F562E43561F56161
:102503008007E5667003756608AB600562E562AA3D
:10251300617002056114F9121E3DF56DC3946140AB
:102523000AE56DD3947A5003536DDF74D0256DF5AE
:102533006DC3940A400CE56D9411406D74F9256DDB
:10254300F56DE56DD395665060436801856C7185C3
:102553006B70856A6F85696EAF667E00E4FCFDABC8
:102563006CAA6BA96AA869121FBFC8ECC8C9EDC9D8
:10257300CAEECACBEFCBE4FCFDFEEB256DF56CEEAA
:102583003AF56BED39F56AEC38F569AF6CAE6BADC6
:102593006AFCAB71AA70A96FA86ED3121F5F5003B8
:1025A30002250C43680402250CE56820E003E4805F
:1025B3002DE56445654563601EAB60E56224FFF964
:1025C300E56134FFFAEBC0E0EAC0E0E9C0E0AB63E9
:1025D300AA64A96512201EE56830E20774FFFFFEB6
:1025E300FDFC22E568AF6CAE6BAD6AAC6930E1030C
:0425F300021F512250
:101FAD00BB010689828A83F0225002F722BBFE0113
:021FBD00F3220D
:101FBF00E88FF0A4CC8BF0A42CFCE98EF0A42CFCC1
:101FCF008AF0EDA42CFCEA8EF0A4CDA8F08BF0A43F
:101FDF002DCC3825F0FDE98FF0A42CCD35F0FCEB9E
:101FEF008EF0A4FEA9F0EB8FF0A4CFC5F02ECD3963
:0F1FFF00FEE43CFCEAA42DCE35F0FDE43CFC22D0
:10200E00FAE6FB0808E6F925F0F618E6CA3AF622D3
:10201E00BB011A89828A83D0F0D0E0F8D0E0F9D0E3
:10202E00E0FAD0E0FBE8C0E0C0F002209C5016E9D8
:10203E00F8D083D082D0E0F9D0E0FAD0E0FBC082B5
:10204E00C083022093BBFE16E9F8D083D082D0E085
:0F205E00F9D0E0FAD0E0FBC082C0830220A522B7
:10206D00D083D082F8E4937012740193700DA3A302
:10207D0093F8740193F5828883E473740293686016
:06208D00EFA3A3A380DF16
:09209300EBF608EAF608E9F62272
:09209C00EBF0A3EAF0A3E9F02245
:0920A500EBF208EAF208E9F2226C
:00000001FF
